:020000021000EC
:10F000004BC0000082C0000080C000007EC0000035
:10F010007CC000007AC0000078C0000076C000000C
:10F0200074C0000072C000004DC500006EC000003A
:10F030006CC000006AC0000068C0000066C000002C
:10F0400064C0000062C0000060C000005EC000003C
:10F0500039C300005AC0000058C0000056C000006C
:10F0600054C0000052C0000050C000004EC000005C
:10F070004CC000004AC0000048C0000046C000006C
:10F0800044C0000042C0000040C000003EC000007C
:10F090003CC000003AC0000011241FBECFEFD0E2F8
:10F0A000DEBFCDBF04B603FE19C08091A0019091D0
:10F0B000A10182349C4D91F484B7877F84BF88E19D
:10F0C0000FB6F89480936000109260000FBE10920B
:10F0D000A1011092A001E0E0F0E0099511E0A0E0AC
:10F0E000B1E0EEE9FEEF01E00BBF02C007900D9228
:10F0F000A239B107D9F721E0A2E9B1E001C01D9220
:10F10000A03AB207E1F731D0C8C67ACF84E0809345
:10F11000E9008091E80085FD0EC08091E8008B77C2
:10F120008093E8008091E80082FDF3CF8EB38111D7
:10F13000F9CF80E008958091F100089593E09093D5
:10F14000E9009091E80095FF03C08093F1000895D5
:10F150009091E8009E779093E8009091E80090FDF0
:10F16000F4CF9EB39111F9CF0895CF93DF9300D0E0
:10F1700000D000D0CDB7DEB784B7877F84BF88E1E9
:10F180000FB6F89480936000109260000FBE90E07C
:10F1900080E80FB6F89480936100909361000FBEF1
:10F1A00011E015BF82E085BF72D410936F0083E039
:10F1B000809381007894F4E08F2EA3E07A2E992436
:10F1C0009394B5E06B2E13E0212E312CAA24A39446
:10F1D000B12C80910001882309F45DC28092E9007E
:10F1E0008091E80082FF55C291DF982F853419F491
:10F1F0001092000107C088E8890F823010F0943522
:10F2000021F484DF8DE09ADF1DC29035D9F39C3460
:10F21000C9F3943711F484E483C0913611F489E57D
:10F22000F2CF913491F472DF182F70DF90E0880FE5
:10F23000991F212F30E0322F2227330F822B932B5F
:10F24000AA2797FDA095BA2FD1C1903711F483E575
:10F25000DACF933559F40AE811E0F80181918F0172
:10F260006DDFF1E001391F07C1F7ECC1963521F4DC
:10F2700081E364DF80E3C7CF933731F482E85EDF58
:10F2800087E95CDF8EE1BFCF953601F580E090E045
:10F29000DC01FC01A0935B0070925700E89507B673
:10F2A00000FCFDCFFC01A0935B0060925700E89545
:10F2B00007B600FCFDCF9F5FAF4FBF4F811520EF1A
:10F2C000920721E0A207B10521F79CCF9C3651F4AB
:10F2D0001DDF809599E0E1E0F0E0082E9093570063
:10F2E000E89590CF923719F489E0F50110C0963473
:10F2F00021F489E0E0E0F0E00AC09E3419F489E0EE
:10F30000F10105C0913539F489E0E2E0F0E0809345
:10F310005700849178CF923631F489E50FDF81E090
:10F320000DDF80E070CF923419F0973609F0E2C01B
:10F330009983ECDE482E512C542C4424E7DE482AD5
:10F34000E5DE182F8BEB810F9981823010F08FE36F
:10F350005ACF973609F04AC081E180935700E8956B
:10F360009201512C2115310509F46CC1C090920114
:10F37000D0909301E0909401F0909501D701C601DF
:10F380001634D1F48529ABBFFC01879129833A83D8
:10F39000D5DE29813A81552069F0F2E0CF0ED11CEB
:10F3A000E11CF11CC0929201D0929301E092940171
:10F3B000F0929501592417C0B695A7959795879512
:10F3C00029833A8354D5BADE82E0C80ED11CE11CF1
:10F3D000F11CC0929201D0929301E0929401F092BC
:10F3E00095013A81298121503109BCCFC090920109
:10F3F000D0909301E0909401F0909501163429F09B
:10F400005E824D82412C512C3DC0F601E0925B00A2
:10F4100070925700E89507B600FCFDCFF1CF163487
:10F4200009F038C0552099F1409192015091930113
:10F43000609194017091950149835A836B837C8319
:10F4400065DE242D30E0382B49815A816B817C8127
:10F450000901FA0160935B0090925700E89511242E
:10F460004E5F5F4F6F4F7F4F4093920150939301D8
:10F4700060939401709395015924ED81FE81319739
:10F48000FE83ED838D819E81892B49F626C03EDE69
:10F49000482EF2CF3BDE682F80919201909193012C
:10F4A000A0919401B0919501B695A79597958795F0
:10F4B000E6D48091920190919301A0919401B09132
:10F4C00095010296A11DB11D809392019093930125
:10F4D000A0939401B0939501D0CF163409F092CE49
:10F4E000F601E0925B0060925700E89507B600FCD9
:10F4F000FDCF88CE933499F4C0909201D0909301BF
:10F50000E0909401F090950101DE90E00C01F6018D
:10F51000E0925B0090925700E895112473CE9336E9
:10F5200019F5C0909201D0909301E0909401F09071
:10F530009501ECDDB701A601416090E00C01FA01F4
:10F5400060935B0090925700E895112492E0C90EF9
:10F55000D11CE11CF11CC0929201D0929301E09267
:10F560009401F09295014ECE9D3691F480919201D6
:10F5700090919301A0919401B0919501FC01A09309
:10F580005B0060925700E89507B600FCFDCF3ACECD
:10F59000923581F48091920190919301A091940110
:10F5A000B0919501ABBFFC0107911691812FC6DD8B
:10F5B000802F29CE943419F5A9DD682F809192010E
:10F5C00090919301A0919401B0919501B695A79562
:10F5D0009795879554D48091920190919301A09131
:10F5E0009401B09195010296A11DB11D80939201E5
:10F5F00090939301A0939401B093950103CE943618
:10F60000F1F4C0909201D0909301E0909401F090B9
:10F610009501D701C601B695A7959795879527D4EB
:10F620008DDDE2E0CE0ED11CE11CF11CC0929201F6
:10F63000D0929301E0929401F092950103C09B3126
:10F6400009F085CE7092E9009091E8008091E80081
:10F650008E778093E80095FD11C08091E80080FDD1
:10F6600004C08EB38111F9CF14C08091E8008E7769
:10F670008093E80003C08EB3882359F08091E8009E
:10F6800080FFF9CF8092E9008091E8008B7780932A
:10F69000E800D2D39ECD8091E00081608093E000AD
:10F6A00082E49CED9093A1018093A0012CE088E17D
:10F6B00090E00FB6F894A895809360000FBE209359
:10F6C0006000FFCF1F920F920FB60F9211240F9080
:10F6D0000FBE0F901F90189542E061EC82E064D15C
:10F6E00042E161E883E060D142E160E884E05CC12E
:10F6F00080919801982F9F77913299F59091990177
:10F70000913229F0923229F1903259F510C0813AA4
:10F7100041F58091E800877F8093E80067E070E022
:10F7200081E091E0AAD08091E8008B770FC0813210
:10F73000C1F48091E800877F8093E80067E070E083
:10F7400081E091E0F5D08091E8008E778093E80029
:10F750000895813231F48091E800877F8093E8003A
:10F7600037C10895292F30E02230310539F0233098
:10F77000310549F02130310561F410C08EE390E08D
:10F780002AE331E01EC0882371F0813089F0823095
:10F79000A1F080E090E020E030E013C082E190E052
:10F7A00028E731E00EC084E090E026E331E009C0B4
:10F7B00088E190E02CE131E004C082E190E028E0B3
:10F7C00031E0FA0131832083089507B600FCFDCFB4
:10F7D000F999FECF23E0FB0180935B002093570053
:10F7E000E89507B600FCFDCF81E180935700E895CE
:10F7F000089507B600FCFDCFF999FECF25E0FB0187
:10F8000080935B0020935700E89507B600FCFDCF7E
:10F8100081E180935700E895089507B600FCFDCF7D
:10F82000F999FECF21E00A01FB0180935B00209350
:10F830005700E8951124089521E2FC012093570018
:10F840008491089529E0FC01209357008491089544
:10F85000E1E0F0E089E0809357008491089507B6D5
:10F8600000FCFDCFF999FECF809599E0E1E0F0E052
:10F87000082E90935700E895089520919E013091AD
:10F880009F012617370748F06115710539F420915B
:10F89000E8002E772093E80001C0B901FC0120E0C8
:10F8A0006115710591F18EB38823E1F18530E1F1A5
:10F8B0008091E80083FD3AC08091E80082FF06C095
:10F8C0008091E80082FF24C080E008958091E800E4
:10F8D00080FFE6CF8091F2009091F30061157105F1
:10F8E00051F08830910538F421912093F100615056
:10F8F00071090196F3CF21E0089709F020E080918B
:10F90000E8008E778093E800CBCF2111CCCFD8CF01
:10F910008EB3882339F0853039F08091E80083FF79
:10F92000CFCF04C082E0089583E0089581E0089578
:10F930006115710529F42091E8002B772093E800E8
:10F940006115710521F12EB3222351F1253051F1BA
:10F950002091E80023FD20C02091E80022FFF3CF92
:10F96000FC01CF012091F2003091F300232B19F319
:10F970008091F1008193CF0161507109611571058A
:10F9800081F7D9CF8EB3882359F0853059F0809113
:10F99000E80080FFF7CF02C081E0089580E008957D
:10F9A00082E0089583E008958F708093E900EBEE84
:10F9B000F0E0808181608083EDEEF0E01082609362
:10F9C000EC0040838091EE00881F8827881F0895EF
:10F9D0008091980187FD05C08091E80080FF0DC0EF
:10F9E00010C08091E80082FD04C08EB38111F9CF70
:10F9F00008958091E8008B7707C08EB38111ECCF1A
:10FA000008958091E8008E778093E80008950F9321
:10FA10001F93CF93DF9349D050D0C8EDD0E08881B9
:10FA20008F77888388818068888388818F7D8883A9
:10FA3000E7EDF0E080818068808319BC1EBA1092E7
:10FA4000960100EE10E0F80180818B7F8083888131
:10FA50008160888342E060E080E0A6DFE1EEF0E0D4
:10FA600080818E7F8083E2EEF0E080818160808300
:10FA7000808188608083F80180818E7F8083888187
:10FA800080618883DF91CF911F910F910895E8EDF8
:10FA9000F0E080818F7E8083E7EDF0E080818160FF
:10FAA000808381E080939701B2CFE8EDF0E0808120
:10FAB0008C7F80831092E20008951092DA001092F9
:10FAC000E10008951F920F920FB60F9211240BB60A
:10FAD0000F922F933F934F935F936F937F938F93E7
:10FAE0009F93AF93BF93EF93FF938091DA0080FFD2
:10FAF0001BC08091D80080FF17C08091DA008E7FF4
:10FB00008093DA008091D90080FF0BC084E189BD29
:10FB100086E189BD09B400FEFDCF81E08EBB8BD1AB
:10FB200003C019BC1EBA87D18091E10080FF17C0C5
:10FB30008091E20080FF13C08091E2008E7F80936D
:10FB4000E2008091E20080618093E2008091D80021
:10FB500080628093D80019BC85E08EBB6CD1809107
:10FB6000E10084FF2EC08091E20084FF2AC084E17E
:10FB700089BD86E189BD09B400FEFDCF8091D80022
:10FB80008F7D8093D8008091E1008F7E8093E1008B
:10FB90008091E2008F7E8093E2008091E20081609C
:10FBA0008093E20080919601882311F084E007C0E1
:10FBB0008091E30087FF02C083E001C081E08EBB3B
:10FBC0003AD18091E10083FF21C08091E20083FF60
:10FBD0001DC08091E100877F8093E10082E08EBBB1
:10FBE000109296018091E1008E7F8093E1008091D8
:10FBF000E2008E7F8093E2008091E200806180933A
:10FC0000E20042E060E080E0CFDE15D1FF91EF91AD
:10FC1000BF91AF919F918F917F916F915F914F9124
:10FC20003F912F910F900BBE0F900FBE0F901F9022
:10FC300018951F93CF93DF9300D0CDB7DEB7E8E9D7
:10FC4000F1E08091F100819381E0E03AF807C9F793
:10FC50004FDD8091E80083FFDAC090919801809198
:10FC60009901853009F465C030F4813059F168F0AC
:10FC7000833041F1CCC0883009F49CC0893009F44C
:10FC8000ABC0863009F0C3C075C0903881F092389F
:10FC900009F0BDC080919C018F708093E900909124
:10FCA000EB0095FB992790F91092E90001C090E0D4
:10FCB0008091E800877F8093E8009093F100109294
:10FCC000F10083C0292F2D7F09F0A1C0923009F0E7
:10FCD0009EC090919A01911126C020919C012F7095
:10FCE00009F495C02093E9009091EB0090FF1BC0B0
:10FCF000833021F48091EB00806213C08091EB008F
:10FD000080618093EB0081E090E0022E01C0880FBB
:10FD10000A94EAF78093EA001092EA008091EB00DF
:10FD200088608093EB001092E9008091E800877F63
:10FD30004FC091116CC010919A011F778091E30020
:10FD40008078812B8093E3008091E800877F809307
:10FD5000E8003EDE8091E80080FFFCCF8091E30068
:10FD600080688093E300112311F083E001C082E0FA
:10FD70008EBB4DC09058923008F049C0AE014F5F25
:10FD80005F4F60919C0180919A0190919B01EADC08
:10FD9000009709F43CC02091E800277F2093E800F9
:10FDA000BC0189819A8169DD8091E8008B7780931D
:10FDB000E8002DC0903859F58091E800877F809346
:10FDC000E800809196018093F1008091E8008E77A1
:10FDD0008093E800FDDD1BC0911119C090919A013C
:10FDE0009230A8F48091E800877F8093E800909398
:10FDF0009601EEDD80919601811104C08091E300AF
:10FE000087FF02C084E001C081E08EBB65DC809189
:10FE1000E80083FF0AC08091E800877F8093E800B4
:10FE20008091EB0080628093EB000F900F90DF9148
:10FE3000CF911F9108950895CF938EB38823A9F091
:10FE40008091E9008F709091EC0090FF02C090E8E3
:10FE500001C090E0C92FC82B1092E9008091E80002
:10FE600083FDE7DECF70C093E900CF910895F99943
:10FE7000FECF92BD81BDF89A992780B50895262FAF
:10FE8000F999FECF1FBA92BD81BD20BD0FB6F8947F
:0EFE9000FA9AF99A0FBE01960895F894FFCFE2
:10FE9E00010000000000000812034C00550046004F
:10FEAE0041002000430044004300000018034400BA
:10FEBE00650061006E002000430061006D0065006A
:10FECE007200610000000403090409023E000201F1
:10FEDE000080320904000001020201000524001016
:10FEEE00010424020205240600010705820308000E
:10FEFE00FF09040100020A000000070504021000B9
:10FF0E00050705830210000512011001020000080A
:10FF1E00EB034A200001010200014C5546414344C7
:02FF2E0043008E
:10FFA00014CC27CC3ACC48CC4DCC52CC58CC08956C
:08FFB0000895089508950895D5
:10FFE000DFCFDFCFDFCFDFCFDFCFDFCFDFCFDFCFA1
:08FFF000DFCFDFCFDFCFDFCF51
:08FFF80000F0010000DFFBDC5A
:040000031000F000F9
:00000001FF
